:020000040800F2
:10000000001800200508000835050008390500081B
:1000100000000000000000000000000000000000E0
:10002000000000000000000000000000350500088E
:10003000000000000000000035050008350500083C
:1000400035050008350500083505000835050008A8
:100050003505000835050008350500083505000898
:100060003505000835050008350500083505000888
:100070003505000835050008350500083505000878
:100080003505000835050008350500083505000868
:100090003505000835050008350500083505000858
:1000A0003505000835050008350500083505000848
:1000B00035050008350500083505000899010008D8
:1000C000284B10B51A88284B12041B881A43274B5B
:1000D000198849084900885A254908801988023139
:1000E00089B21980198849084900885A214908802D
:1000F0001988023189B21980198849084900885A3B
:100100001D49088019881D48023189B21980198853
:1001100049084900895A1A4A11801A881949023235
:1001200092B21A801C880288944213D902881C88D3
:100130000832121B92B20A80028892B21A801249C7
:10014000124B0A881343124A1A40302353409BB281
:100150000B8010BD0F4804881A889442E6D3082308
:100160000B80ECE70C6000400A6000400460004037
:100170004C6000404E600040506000400260004013
:10018000526000401A600040005C00408080FFFF29
:10019000BF8FFFFF006000409449F8B50B88944C76
:1001A000002B3AD00A88934B9A4234D1002302257F
:1001B000914A924F1380924A1380924A1380924A36
:1001C0001380924A1380924AD08FA843D087D08F51
:1001D000013DA843D0878F481735FB8705808E489F
:1001E000343505808D480835058080258C486D01A3
:1001F000058080258B4805808020FB878A4B000680
:1002000023808A4B18608023D08FDB000343D38781
:10021000874B884A1A8000230B8023881BB2002B4F
:1002200000DBC4E02388844A774F134080221343C5
:10023000238023881B0500D49CE0804D7F232A78EF
:1002400011009943714B1980E9886B4B198000218B
:100250006C4B19803B88FF318B4313433B806023F9
:100260001A4208D08022764B12051B8828009B1862
:100270009847634B188060232A78134052B2002AB3
:100280004DDA002B14D16A78062A0FD16A88110A38
:1002900002291AD003291BD0012920D1694B12262B
:1002A000694A99B21180694A1B0C1380544B1E8015
:1002B0002288674B1343674A1A40C0239B0153406F
:1002C0009BB22380FFF7FCFE47E05E4B1233E6E76C
:1002D000D2B2012A0FD0002A03D0022A15D01E0064
:1002E000E4E7584B584A243399B21180574A1B0C03
:1002F00013800426DAE7534B534A283399B211800E
:10030000524A1B0C1380544ED0E74E4B4E4A7C335E
:1003100099B211804D4A1B0C1380504EC6E7002B3A
:1003200009D16B78052B06D13A886B88D2B21B02B3
:1003300013439BB23B8000212388494A1340494A1A
:1003400013439BB22380484B198023881A43474BA1
:100350001A40474B5A4092B22280284BDB8F5B05F4
:1003600007D580222F4B1A800023244AD3872E4B97
:100370002380F8BD60213B880B40402BEDD13B88AA
:100380001342EAD1264A3B4B2C481B881188802215
:1003900012059B18C9B298472288324B13432D4A45
:1003A0001A40C0239B0153409BB22380D5E7802293
:1003B00023881342D1D023882F490B408021090282
:1003C0000B432380114B1B88934200D17AE7FF2017
:1003D0000D4B19888143C0D01988090A0A43114975
:1003E0000A801A8802401A80B7E7C0460E600040B3
:1003F000005C00403CA5000000600040065C00403E
:100400000260004004600040066000400860004058
:10041000025C0040505C0040186000401C600040DE
:100420001E6000404C5C00402032000000E100E013
:10043000585C00400080FFFF8F0F000054600040B8
:10044000106000407C0400080A6000400C6000401E
:100450008081FFFF8FBFFFFF2A0300001E03000003
:100460008F8EFFFF8080FFFF1A600040BFBFFFFF3D
:1004700030300000126000400F8FFFFF12010002B9
:10048000FF000008C016DC0503020102000109029A
:100490001200010100803209040000000000000089
:1004A000040309042A0349006E00660069006E0017
:1004B0006900740065004E00650073004C0069001F
:1004C0007600650073002E0063006F006D00000071
:1004D000000000000000000000000000000000001C
:1004E000000000000000000000000000000000000C
:1004F00000000000000000001E0349004E004C00F8
:10050000200052006500740072006F002D00500042
:1005100072006F0067000000000000000000000093
:1005200000000000000000000000000000000000CB
:1005300000000000FEE7FFFF004801E02301ADDE00
:10054000FEE7C04602B4714649084900095C49000B
:100550008E4402BC7047C046411D000000616561C9
:1005600062690001130000000536532D4D00060C92
:10057000074D09011901FFFF03B471464908400006
:100580004900095A49008E4403BC7047411D0000D0
:100590000061656162690001130000000536532D9A
:1005A0004D00060C074D09011901FFFF70470A4B6A
:1005B0000A4A10B55A600A4A5A600122DC6814429D
:1005C000FCD11A6101220180D9681142FCD120229C
:1005D000DA6060321A6110BD0020024023016745D5
:1005E000AB89EFCDFF2370B53C4C23804378C588A1
:1005F000102B00D06FE0C37881888078384E0138A6
:100600007269082800D964E0FFF79CFF0563632B3B
:100610003B3149515F008B1E8E227D2B19D8314B07
:100620007360314B73600123F2681A42FCD10223DC
:100630003361802389021B05C9184223716133612C
:10064000C046413BF2681A40FCD12023F36060337E
:1006500033612270254BA2B2240CE8B25A819C81EE
:1006600070BD58001018FFF7A2FF0022F1E78E229C
:10067000012BEED8180480231B05C01840181C4914
:10068000F1E7042363707369A37073691B0AE37055
:1006900073691B0C237173691B0E6371E5E70223F9
:1006A00063701388A37013881B0AE370DDE78E2242
:1006B000012BCED880221B0412059B185918022347
:1006C00063700B88A3700B88EEE70A4B0A4ADA6066
:1006D000CBE78B22BDE780232370BBE7F806002021
:1006E0000020024023016745AB89EFCD0060004048
:1006F000FFFF000000ED00E00400FA05FFFFFFFF30
:10070000FFFFFFFFFFFFFFFFFFFFFFFFFFFFFFFFF9
:10071000FFFFFFFFFFFFFFFFFFFFFFFFFFFFFFFFE9
:10072000FFFFFFFFFFFFFFFFFFFFFFFFFFFFFFFFD9
:10073000FFFFFFFFFFFFFFFFFFFFFFFFFFFFFFFFC9
:10074000FFFFFFFFFFFFFFFFFFFFFFFFFFFFFFFFB9
:10075000FFFFFFFFFFFFFFFFFFFFFFFFFFFFFFFFA9
:10076000FFFFFFFFFFFFFFFFFFFFFFFFFFFFFFFF99
:10077000164B174A9BB21382164B9BB253826846A4
:100780001C300F4A0F4B0430043001681140C91A65
:10079000FAD1094A094B043801681140C91AF2D14B
:1007A0007B460A3303600438013303600CE00A4BD4
:1007B0000A4A1A60FBE7C0460000FFFF000000087D
:1007C000FFFFFF0F0000000100207047E505000853
:1007D00000600040AD05000800300040AAAA0000FB
:1007E000FFFFFFFFFFFFFFFFFFFFFFFFFFFFFFFF19
:1007F000FFFFFFFFFFFFFFFFFFFFFFFFFFFFFFFF09
:10080000FFFFFFFF09490A4A0A4B9B1A03DD043B1D
:10081000C858D050FBDC0849084A0020521A02DDB3
:10082000043A8850FCDC03F029F8000070560008F8
:100830000000002030040020300400203807002091
:1008400070B50E4B1A68537A55685C18E4B2A3422F
:100850000ED1537A0A48CB1853720378591AC9B289
:1008600001700020814202D198230130D37070BD05
:1008700006780130EE540133DBB2E8E7940400203F
:1008800098040020FF23F0B5C04C85B02380837905
:100890000700009340780138102801D901F0F4FDD9
:1008A000FFF76AFE1100D405B108EC09980CF20DAF
:1008B000DE0D2F0BB40B1F0C790C460A940ACF0ADD
:1008C000FE0AF20D7C0CB878BA888C231D2826D835
:1008D000FFF752FE1E0028001E011802E4028303E7
:1008E0000E04CA04E604F204FA0402050B0514051A
:1008F00022052A0532053A05AA05AA05AA054A05D0
:100900005F057605CC02D8023F058D059605A10549
:10091000B0239F4A5B0351690B435361002323704B
:1009200000F0D8FE152A01D900F081FD1000FFF774
:1009300023FE160023002E007E05390044004F00E0
:100940007E055C006900730080007E057E058D00D9
:100950009A00A700B400C100CE00D800E2009023A6
:10096000DB051A688B490A401A608022D968520355
:100970000A43DA600023D2E790230122DB051968DD
:1009800091431960D9680A43DA600023C7E79023CE
:100990000422DB05196891431960D9680A43DA60BB
:1009A0000023BCE790231022DB05196891431960EE
:1009B000D9680A43DA600023B1E790234022DB05BF
:1009C000196891431960D9680A43DA600023A6E7E1
:1009D0009023DB051A6870490A401A608022D968A2
:1009E000D2040A43DA60002399E79023DB051A68F2
:1009F0006A490A401A608022D96852010A43DA60C3
:100A000000238CE70422664B196891431960D9686A
:100A10000A43DA60002382E79023DB051A68614904
:100A20000A401A608022D968D2050A43DA6000239E
:100A300075E79023DB051A685B490A401A6080223B
:100A4000D968D2020A43DA60002368E79023DB0505
:100A50001A6856490A401A608022D96852000A432F
:100A6000DA6000235BE79023DB051A6850490A40EF
:100A70001A608022D968D2000A43DA6000234EE768
:100A80009023DB051A684B490A401A608022D96816
:100A9000D2010A43DA60002341E79023DB051A689C
:100AA0003D490A401A608022D968D2040A43DA60BC
:100AB000002334E79023DB051A683F490A401A6097
:100AC0008022D96852050A43DA60002327E7012211
:100AD000334B196891431960D9680A43DA600023DF
:100AE0001DE71022354B196891431960D9680A43F4
:100AF000DA60002313E79023DB051A682C490A40CB
:100B00001A608022D968D2000A43DA60002306E71F
:100B1000152A01D900F08EFC1000FFF72DFD1600FC
:100B200021002C008B0451005C0067008B047200D4
:100B30007D00870092008B048B049D00A800B30009
:100B4000BE00C900D400DE00E8009023DB05196870
:100B5000104801401960DA680240DA600023DEE6DE
:100B600090230121DB051A688A431A60DA688A43F8
:100B7000DA600023D3E690230421DB051A688A4358
:100B80001A60DA688A43DA600023C8E600070020AA
:100B900000100240FFFFEFFFFFFFFFFBFFEFFFFF33
:100BA00000040048FFFFFFBFFFFFFBFFFFFEFFFF4A
:100BB000FFFBFFFFFFBFFFFFFFFFFFEF000C004841
:100BC00090231021DB051A688A431A60DA688A4389
:100BD000DA600023A3E690234021DB051A688A43EC
:100BE0001A60DA688A43DA60002398E69023DB050E
:100BF0001968CE4801401960DA680240DA600023C3
:100C00008DE69023DB051968C94801401960DA6850
:100C10000240DA60002382E60421C64B1A688A4348
:100C20001A60DA688A43DA60002378E69023DB05ED
:100C30001968C14801401960DA680240DA6000238F
:100C40006DE69023DB051968BC4801401960DA683D
:100C50000240DA60002362E69023DB051968B84899
:100C600001401960DA680240DA60002357E69023F9
:100C7000DB051968B34801401960DA680240DA60A0
:100C800000234CE69023DB051968AF48014019604A
:100C9000DA680240DA60002341E69023DB05196838
:100CA000A24801401960DA680240DA60002336E6A3
:100CB0009023DB051968A54801401960DA680240F5
:100CC000DA6000232BE601219A4B1A688A431A60E6
:100CD000DA688A43DA60002321E610219C4B1A6807
:100CE0008A431A60DA688A43DA60002317E69023A1
:100CF000DB051968934801401960DA680240DA6040
:100D000000230CE6152A00D997E31000FFF734FC06
:100D100016001F00270095032F0037003F009503A2
:100D20004800510058006100950395036A00730064
:100D30007C0085008E0097009E00A50090228023F5
:100D4000D20511685B030B4313600023E7E5902293
:100D50000123D20511680B4313600023DFE59022C5
:100D60000423D20511680B4313600023D7E59022BA
:100D70001023D20511680B4313600023CFE59022A6
:100D80004023D20511680B4313600023C7E590226E
:100D90008023D2051168DB040B4313600023BEE5FA
:100DA00090228023D20511685B010B43136000235E
:100DB000B5E504235F4A11680B4313600023AEE5D9
:100DC00090228023D2051168DB050B4313600023BA
:100DD000A5E590228023D2051168DB020B43136046
:100DE00000239CE590228023D20511685B000B4311
:100DF0001360002393E590228023D2051168DB0065
:100E00000B43136000238AE590228023D2051168EA
:100E1000DB010B431360002381E590228023D20580
:100E20001168DB040B431360002378E590228023D4
:100E3000D20511685B050B43136000236FE50123A6
:100E40003C4A11680B431360002368E51023404AB5
:100E500011680B431360002361E590228023D205C3
:100E60001168DB000B431360002358E58D23082A2B
:100E700000D054E590224023D20551680B435360C3
:100E800000234CE58D23082A00D048E5902240211C
:100E9000D20553688B435360002340E5152A00D9DF
:100EA000CEE21000FFF768FB16001D002300CC0205
:100EB00029002F003500CC023C0056005B00620088
:100EC000CC02CC0269006F0075007B0082008900B3
:100ED0008E00930090238022DB05D2009A620023CB
:100EE0001DE590230122DB059A62002317E590237C
:100EF0000222DB059A62002311E590230422DB0520
:100F00009A6200230BE590230822DB059A620023F6
:100F100005E590238022DB0592019A620023FEE41E
:100F200090234022DB059A620023F8E4FFFFFFFBD9
:100F3000FFEFFFFF00040048FFFFFFBFFFFFFBFFC5
:100F4000FFFEFFFFFFFBFFFFFFBFFFFFFFFFFFEF06
:100F5000000C00480222CD4B9A620023DFE490236C
:100F60008022DB0512029A620023D8E490238022BB
:100F7000DB0592009A620023D1E490231022DB0566
:100F80009A620023CBE490232022DB059A6200239F
:100F9000C5E490238022DB059A620023BFE49023FE
:100FA0008022DB0592019A620023B8E4902380221C
:100FB000DB05D2019A620023B1E40122B34B9A62AD
:100FC0000023ACE40422B24B9A620023A7E49023EE
:100FD0002022DB059A620023A1E4152A00D932E21F
:100FE0001000FFF7C9FA16001D0023003002290087
:100FF0002F00350030023C00420047004E00300216
:10100000300255005B00610067006E0075007A00D9
:101010007F0090238022DB05D2009A6100237EE4CA
:1010200090230122DB059A61002378E490230222B9
:10103000DB059A61002372E490230422DB059A61A8
:1010400000236CE490230822DB059A61002366E408
:1010500090238022DB0592019A6100235FE49023B4
:101060004022DB059A61002359E40222874B9A61F2
:10107000002354E490238022DB0512029A610023AE
:101080004DE490238022DB0592009A61002346E420
:1010900090231022DB059A61002340E49023202254
:1010A000DB059A6100233AE490238022DB059A61F4
:1010B000002334E490238022DB0592019A6100230F
:1010C0002DE490238022DB05D2019A61002326E4DF
:1010D00001226E4B9A61002321E404226C4B9A6139
:1010E00000231CE490232022DB059A61002316E4F0
:1010F00002236370152A00D9B1E01000FFF722FA2D
:101100000B151EAF273039AF434C545DAFAF67703E
:1011100079828C969EA690238022DB051B69D200E3
:10112000134063800023FFF7FAFB90230122DB05C5
:101130001B69134063800023FFF7F1FB9023022219
:10114000DB051B69134063800023FFF7E8FB902356
:101150000422DB051B69134063800023FFF7DFFBDC
:1011600090230822DB051B69134063800023FFF7EF
:10117000D6FB90238022DB051B699201134063801C
:101180000023FFF7CCFB90234022DB051B691340B3
:1011900063800023FFF7C3FB02223C4B1B69134013
:1011A00063800023FFF7BBFB9023DB051B69DB0B90
:1011B000DB0363800023FFF7B2FB90238022DB0573
:1011C0001B699200134063800023FFF7A8FB902364
:1011D0001022DB051B69134063800023FFF79FFB90
:1011E00090232022DB051B69134063800023FFF757
:1011F00096FB90238022DB051B691340638000234C
:10120000FFF78DFB90238022DB051B6992011340C1
:1012100063800023FFF783FB90238022DB051B699B
:10122000D201134063800023FFF779FB0122174BA3
:101230001B69134063800023FFF771FB0422144BEA
:101240001B69134063800023FFF769FB9023202272
:10125000DB051B69134063800023FFF760FB00235D
:1012600063708D33FFF75BFB80230A4ADB02516911
:101270000B435361054B08491A680A401A60D96844
:10128000064A0A43DA600023FFF749FB00040048DE
:10129000000C004800100240FFFFAAAA00005555AC
:1012A000C84BC9491A680A401A60D968C74A0A4334
:1012B000DA600023FFF733FBC24AC34913680B40CF
:1012C00013600023FFF72BFBBE4AC04B11680B4392
:1012D00013600023FFF723FBBA4912024B69DBB20C
:1012E0001A434A610023FFF71AFBB64B1B691B0A1E
:1012F000A370012363700023FFF711FB8023B44A1E
:101300001B0351690B435361B24AB34B11680B4342
:1013100013600023FFF703FBAE4AAF4BD1680B43CA
:10132000D3600023FFF7FBFAAA4AAC4913680B40CD
:1013300013600023FFF7F3FAA64AA74B11680B438B
:1013400013600023FFF7EBFAA24B5A610023FFF76B
:10135000E6FA012363709F4B1A69A2701B691B0A8E
:10136000E3700023FFF7DBFAC023994ADB025169DF
:101370000B435361934A9A4B11680B4313609022BD
:10138000A023D20511685B030B4313600023FFF712
:10139000C6FA8C4A924BD1680B43D3609023A021AC
:1013A000DB05D86849030143D96011688D480140C5
:1013B00011601A688C490A401A600023FFF7AFFADF
:1013C000FF258048930041692B40884DD200294079
:1013D0000B4343619021C020C905C0004B69024006
:1013E000834803401A434A610023FFF798FA01211A
:1013F000744B1A680A431A6099620023FFF78FFA48
:101400000122704B196891431960D9680A43DA6068
:101410000023FFF784FA6F4B5A610122694B9A61EE
:101420009A620023FFF77BFA0023FFF778FA8D23F7
:10143000FFF775FA8D23FFF772FA8D23FFF76FFA26
:101440008D23FFF76CFA8D23FFF769FABD78BB880F
:10145000052D00D1F1E135D8022D00D185E107D865
:10146000002D00D130E1012D00D13BE196252FE187
:10147000032D00D162E2042DF8D1DBB29825012BB7
:1014800000D025E190225B4BD2051A6006220A218A
:10149000594B1A704B4B594A1360594A1170594AAB
:1014A00001311360584A1170584A13600C22584B8E
:1014B0001A70B023464A5B0351690B43536101F034
:1014C000A5FEAEE1082D00D111E200D9A2E0062D63
:1014D00000D1CEE1072DC9D101F064FF9023012492
:1014E000DB051A68384F22431A6010229C61196884
:1014F0000A4304211A60802299611868D2010243CC
:101500001A6080229A6180221868520102431A6090
:1015100040229A6118680143196002219961196893
:101520002B480A431A6008229A61802241691203FB
:101530000A43284942610D68274A2A430A60214A22
:10154000156825431560842594624D6100259461DA
:1015500094624D6180211C68C90521431960802176
:101560000902996280214469C902214341611168DD
:1015700039401160D66815490E43D6601468194E7B
:101580003C401460D4682143D160C0214469C90241
:10159000214341611068124908431060A0201C6873
:1015A000400304431C601468344014601C680E4EF1
:1015B00034401C60D4682143D160DA680243DA60A9
:1015C00086E0C04600040048FFFFAAAA0000555567
:1015D000001002400008004855555555AAAAAAAA6D
:1015E00050550000AFAAFFFFFFFFEBFF03FF000015
:1015F000FFF9000024070020280700201C07002016
:10160000200700202C0700203007002014070020AE
:10161000180700200A2D00D1FAE000D203E1802D46
:1016200000D023E79023012540208026DB0565704C
:1016300098621A68760132431A60C046D2491C6922
:101640001A6804400A401A60DA680A40DA60F02238
:10165000002C36D11A680A401A60DA683243DA6020
:101660001A6994461A690192C0461A690292C046E4
:10167000C0461A690392C046C046C0461F69C046AC
:10168000C046C046C0461E691A680A401A60DA6839
:101690001140D96063462200034212D1019B2A0007
:1016A00003420ED10299023201420AD10399033258
:1016B000014206D10432074203D1D632064200D09D
:1016C000D13AB24B9A70ACE0B14A137001F06AFEA5
:1016D000AE4C2570AF4B0098A2B2240C5A819C816D
:1016E00005B0F0BD01F05EFE9023DB051A682A43C9
:1016F0001A6080229D61196852030A431A60802291
:101700000421D2009A621A680A431A6002229A617E
:1017100018680E3202431A604022996119680A4320
:101720001A6008229A6180239B49DB024A699B4D1B
:1017300013439B4A4B6113682B401360D468994B49
:101740001C43D460106828401060D0680343D36005
:1017500080234A691B0313434B61934B934A1968D7
:101760000A431A6000255D61B2E701F01BFE902379
:101770000121DB051A6888480A431A601022996122
:101780001968864E0A431A60042240219A611A6839
:101790000A431A6008229A618022996119685201ED
:1017A0000A431A6080224169D2020A437C4942619D
:1017B0000A6832400A60CD687A4A1543CD600C68E9
:1017C00034400C60CC682243CA6080224469120312
:1017D00022434261744A754C15682C4300251460FD
:1017E0005561C0224469D202224342610868704AAE
:1017F00002430A60A0221868520302431A606D482F
:101800004A6902404A615A696B490A405A615FE776
:1018100090238022DB051968D2010A431A608022D6
:101820009A61002554E790238022DB051968D201D4
:101830000A431A6080229A62F3E701F0B3FD902315
:101840000121DB051A680A431A60102299611968A0
:101850000A431A60042240219A611A680A431A60F6
:1018600008229A6180221868520102431A60996125
:1018700059E701F097FD90230121DB051A68474DD8
:101880000A431A601022996119680A431A600422F7
:101890009A6119683C3211431960082199619A6272
:1018A0009A6180233C49DB024A6913433C4A4B61FD
:1018B00013682B401360D4683A4B1C43D460106803
:1018C00028401060D0680343D36080234A691B031B
:1018D00013434B61344B354A19683848114319603A
:1018E000196801401960D9680A43DA603AE701F0E3
:1018F00059FD90230121DB051A680A431A6004226E
:101900009961196811431960196811431960102110
:1019100018680143196040219A611A680A431A60E5
:1019200080229D611868520102431A6099618023E8
:10193000194A1B0351690B435361CBE7DBB2022BFE
:1019400042D00025032B00D1C2E69735012B00D0F1
:10195000BEE68022002510491203486902434A610D
:10196000114A116899431160D1681943D1605168D7
:1019700019435160936111680B431360104B1D7044
:10198000104B1A60A4E6C046FFEFFFFF00070020DF
:10199000080700200060004000100240FFFFAAAAD4
:1019A000000400480000555500080048555555559D
:1019B0005055000003FF0000FFF90000AAAAAAAAE0
:1019C000100700200C070020B023BF4A5B035169B9
:1019D00040200B4353619022D2051368BB490B4052
:1019E00013608023D1685B011943D16051680143C2
:1019F0005160906111680B4308211360B44B19705A
:101A0000B44B1A600DE7BE78F978BD880E2E00D170
:101A1000D2E030D8072E00D1DAE016D8022E00D15D
:101A200098E007D8002E00D186E0012E00D18DE08D
:101A3000A02684E0052E00D1B0E000D981E0042E7C
:101A4000F6D1280001F000FE7EE00A2E00D1AFE0C2
:101A500008D8082E00D1BFE0092EE9D1280001F0F6
:101A6000C1FA71E00C2E00D1BEE000D8ACE0280035
:101A700001F086FA68E0222E70D017D8112E00D11E
:101A8000AEE008D80F2E00D19AE0102ED0D1280059
:101A900001F0D4F958E0202E00D183E000D984E091
:101AA000122EC5D1280001F08FF94DE0822E00D111
:101AB000D1E032D8802E00D19AE000D9C4E0232EA4
:101AC000B6D1854B9D4202D880231B021D4390272F
:101AD00000F0C6FD6B1CFF339BB20193FF057F4BEB
:101AE0007F4E5D6132687F4B00021343FF223360FB
:101AF0007369134018437061C0460823BB6200F04D
:101B0000AFFD08230135BB61019BADB29D42E6D11B
:101B10003368754A1340336016E0852E00D1A0E08B
:101B2000862E00D1A2E0842E00D081E70123280078
:101B3000637000F095FF8CE0280001F0F5F9267045
:101B4000C8E5280001F0CCF90026F8E7280000F0ED
:101B5000A3FFF9E7280001F027F8F5E75F4B022221
:101B60005D6190235E48DB059A6206685D4A090262
:101B70003243026042692DB2D2B211434161002D5D
:101B800001DA01229A62C046C04601229A61921887
:101B90009A610368544A13400360D5E7280000F0B7
:101BA00037FFD1E7514B1D70CEE7514B1D80CBE77E
:101BB000280000F0D7FFC7E7280001F087FDC3E742
:101BC000280001F053FDBFE7280001F09FF8BBE7B4
:101BD000280001F05DF9B7E7280000F0A1FFB3E7A6
:101BE000280001F059F8AFE7280001F013F8ABE73F
:101BF000012190236170DB051868344E3040186075
:101C0000DA6802203240DA608022D2009A6299615A
:101C1000986132484561C046C0462DB29A61002D98
:101C200000DA9962C046C046C046C046C046C046BB
:101C3000902280212A4BD205C9001B6991620121A3
:101C40001B0A9161A3707FE701232800637001F0F4
:101C50009BF8A07078E701232800637000F044FF30
:101C6000F7E701236370214B1B78EBE702236370D6
:101C70001F4B1B88A3701B0AE37065E7B878F978DF
:101C8000BD88AA23062801D9FEF749FEFEF75AFCB3
:101C90000445363D414D3B00FF201149AB004A69E8
:101CA00003401448ED00024013434B619022C021D1
:101CB000D205C90053690D400F490B401D435561C2
:101CC0000023FEF72CFEC04600100240FFEFFFFF8E
:101CD000100700200C070020FF1F0000000800482C
:101CE0000004004800005555FFFFAAAA8C040020FC
:101CF0003604002003FF0000FFF900000022280046
:101D000000F0C6FCDCE70122F9E7280000F006FE3F
:101D1000D6E7280000F0DAFDD2E701230021637046
:101D2000280000F0E5FCA070CAE701216170F7E728
:101D3000BA78BB88002A29D0012A44D1C748F9784B
:101D40004361C020C0011B18C5489BB2834202D822
:101D50009023DB059A62C34BC34A18680902024309
:101D60001A605A69D2B20A435A6190220821D205F8
:101D70009162C046C046C0469161073991611A68B8
:101D8000BA490A401A600023FEF7C9FD0121B34A8F
:101D90006170536190220420D2059062C020C0017E
:101DA0001B18AF489BB2834200D89162C046C04620
:101DB000C046C0460121AB4B1B6991611B0A033130
:101DC0009161A370DFE7AF23FEF7A9FDBD78022D77
:101DD0000BD0032D29D0002D31D10223637001F0E7
:101DE0009BFBA070000AE07073E4BD88A04BF878FC
:101DF0001D80A04BA04A1870984B000219680A4336
:101E000098491A600E68984A32430A605D614A69CF
:101E1000D2B202434A6190220121D20591621A682E
:101E200096490A401A60002553E490230122DB05FD
:101E30009A618C4A8D4913680B401360F3E7B02513
:101E400047E4BA780023012A01D1FEF768FD9A42DF
:101E50001FD0B133022A01D0FEF761FD8421012594
:101E6000BB887E481943426941617E4992B28D61C7
:101E70008D62426104228021134090220902D20522
:101E8000002B03D091610023FEF749FD9162FEF71C
:101E900046FD01236370A933A3701300FEF73FFDD5
:101EA000B878BB88042829D8FEF74CFB182803080B
:101EB0000C00734A13800023FEF731FD180001F077
:101EC000B3F8F8E790230222DB059A61C046C046CA
:101ED000C046C046C046013A9A61ECE79022022310
:101EE0000421D20563709162C046C0465B4B1B69FA
:101EF0009161A3709BB21B0AE370DCE7B223FEF78B
:101F00000EFDBD78FA78B988112D78D007D8012D4B
:101F10004DD0002D0DD0022D5AD082260FE6212D56
:101F200063D0222D67D0122DF7D1022310206370C9
:101F300068E00127534B04261B7810209F40FA438A
:101F4000514B01921D68AF626B6813406B6000F0EB
:101F50007CFBAF616B683B436B60FA20400000F094
:101F600074FBFA20AF626B68019A400013406B600B
:101F700000F06BFBAF616B68013E3B43B6B26B6038
:101F8000002EEAD10436FA2000F05FFBAF626B68E6
:101F9000019AFA2013406B6000F057FBAF616B6849
:101FA000013E3B43B6B26B60002EECD1C7E5354A2B
:101FB000354B12781E689540B56273681020AB43AC
:101FC000736000F042FBB56173682B437360BBE53F
:101FD00001232C4A637012782C4993402A4A9BB201
:101FE0001268002002F0F4F933E601230020637048
:101FF00001F094FB2DE6012310206370F8E7022323
:102000000020637001F0E4FB60809DE5BB78BA8836
:10201000042B1DD007D8022B40D045D8012B12D05D
:102020008723FEF77CFC072B47D003D8052BF7D17D
:10203000174B37E0082B45D0802BF1D101F0E6F8A3
:102040000023FEF76CFC134A1278A2706370F7E766
:10205000114B1B78A3700123F8E7C0460008004825
:10206000FF1F00000004004800005555FFFFAAAA0A
:102070008A0400208804002055555555AAAAAAAA0A
:10208000A0040020100700200C070020040002001C
:10209000E5040020C4040020E6040020C14B1A70AF
:1020A0008322C14B1A70CBE7BE4BBF4D1A708323FE
:1020B0002B7001F01BF92B78CCE7BC4B1A70120A7D
:1020C0005A70BDE7B94B1A78A2705A78E2709A78C4
:1020D0002271DA7862711A79A2715B79E371062351
:1020E000B4E7B878F9780238BA888A23092801D980
:1020F000FEF715FCFEF726FA050A10151C232F3BE8
:102100004048AB4B1A800023FEF709FCA84B1B8804
:102110001B0413439847F6E7FEF72AFB0300FEF77C
:10212000FEFBA448036899B213040B430360EAE77B
:10213000A0490B681B0C1B0413430B60E3E704234B
:1021400063709C4B1B681A0AA370E2701A0C1B0E7A
:1021500022716371D7E7022363705300954A1168B7
:10216000CB181A88A2701B881B0AE370CBE7914B2F
:1021700049001B68CA52C6E78E4953000A68D31843
:1021800002220B606270ECE78A4B49001868411824
:1021900019600A80B7E78823FEF7C1FBBB78BA88CD
:1021A000022B09D0032B0ED0012B10D11304824A2D
:1021B00013600023FEF7B3FB7F490B681B0C1B0465
:1021C00013430B60F5E701227B4B1A60F1E7832391
:1021D000FEF7A5FBBA781300303B2F2B1AD8F878FE
:1021E000032814D8FEF7AEF916180211734B512AC2
:1021F00000D17DE028D8312A57D00FD8002A37D017
:10220000302A4BD0B423FEF78AFB6D4BEFE7B523A2
:10221000FEF785FB6B4BEAE76B4BE8E7332A52D0BE
:102220004AD3502AEED1C022D20022801A7AA2705C
:10223000DA78E2705A7A22719A7A62719A78A27187
:102240005B7CE371FFF746FA7F2A00D984E0702AAD
:102250005DD2602A3CD0612A43D0522AD2D180225A
:102260001B889200A3701B0A2280E370FFF732FAEA
:10227000FF21564BD1540132102AFBD10123514A80
:102280005B425380504A53804C4A53804C4A53809F
:1022900001224F4B1A700023FEF741FBBA88110A46
:1022A000D9721A730023FEF73AFBBA88110A5973E0
:1022B0009A730023FEF733FBBA88110AD9731A7494
:1022C0000023FEF72CFBBA885A740023FEF727FB85
:1022D00080235B002380BB883C4AD35CA370FFF75C
:1022E000F9F980235B0023803A4B1B68DB78F5E724
:1022F000C022D2002280DA7AA2701A7BE2705A7B66
:1023000022719A7B6271DA7BA2711B7C99E72D4B5B
:1023100038785C682F4B1968CB787F2800D9B6E0F5
:102320002D48009D0570002B0FD000200090982BA9
:1023300000D1B2E004E000200090D02B00D1ACE04E
:10234000234B10301870FF2304E0244B19609023B6
:10235000CB706F330093A0E00720104003281AD8F9
:10236000FEF7F0F81C1E0217144B802A01D2FFF76B
:10237000B1F9872A34D97032D2B2072A01D9FFF7CE
:10238000A9F900222270FA789A72BA881A80FFF7A7
:10239000A1F90B4BE9E7B523FEF7C1FA094BE4E7D6
:1023A000094BE2E7C4040020E6040020C504002035
:1023B00034040020300400209C040020600400202D
:1023C00074040020380400204C040020E70400209E
:1023D000A40400209004002098040020940400200D
:1023E000B888F978C6B28D19BE22102D2CDC0432C3
:1023F000002929D0DD78033AFF2D25D19D780132BF
:10240000FF2D21D10022D7B2B94220D82F4D002272
:10241000AC464F01013F1F727701000A6744987074
:10242000DA705A729A721A80DA721A735A739A733D
:10243000DA731A745A745F60254B9D19A8540132DF
:10244000D3B28B42FAD300222270FFF743F9013254
:10245000B7181F4D013FEF5DFF2FD4D0C122F3E726
:10246000BB78002B04D0402B08D0D223FEF757FABC
:102470002370BA88174B1A70FFF72CF980235B0082
:102480002380144B1B7829E78023FEF748FAD82BCA
:1024900000D050E780234C68CB7000234B72CB7880
:1024A000902B01D0FFF716F9712A01D0FFF712F92E
:1024B000094BBA881B6859680A70BA885968120AA9
:1024C0004A705A7A02325A72FFF704F9F80400206F
:1024D000E7040020A404002094040020F0B51C4D63
:1024E000040005A8067868690902C0B2084368615B
:1024F00090200421C00581622900002A01D1013207
:102500008262FF2500204A692D022A401A43114F9A
:102510004A61C046C046C046C046C046C046C046E6
:10252000C046C046C0463A690133120A22544A697D
:10253000DBB22A4001301A43C0B24A61B042E8D946
:1025400090230422DB059A61033A9A61F0BDC046EC
:102550000008004800040048F0B5184C0500606908
:102560000E02C0B23043606180269020F600C005A4
:1025700049B28661002901DA01218162FF26616981
:102580003602314011436161C04600200C4FC04605
:1025900039690132090A29546169D2B231400130E6
:1025A0001143C0B261619842F1D990238022DB05CA
:1025B000D2009A6201229A61F0BDC046000800482C
:1025C00000040048F0B5174C05000E0060691F2993
:1025D00025D8802131430902C0B2014361619021B5
:1025E0000420FF26C9058862616936023140114323
:1025F0006161C04600200C4FC04639690132090AAA
:1026000029546169D2B2314001301143C0B26161D5
:102610009842F1D990230422DB059A61F0BDC0B243
:102620000902DAE70008004800040048002302001D
:102630000002002A04D1002B01D0802318437047E8
:10264000DB43511EDBB20A40F3E70023800080B277
:10265000C046C04601339BB29842F9D17047FFFF94
:1026600030B50722012409490868450D43086B402D
:102670004340C50FDBB26B40013A23404000D2B269
:102680001843002AF1D10860C0B230BD9C0400207C
:10269000134B10B55861134B13481C6809022043B3
:1026A00018605869C0B20143596190210820C905DA
:1026B0008862002A01D101328A62C046C046C04603
:1026C000C046C046C046C046C04690220821D2053A
:1026D0009161073991611A6804490A401A6010BD76
:1026E000000800480004004800005555FFFFAAAA52
:1026F0000F4B58619023DB05002901D101229A621A
:1027000004229A62C046C046C046C046C046C04683
:10271000C046C046C046C046C046C046C046054941
:1027200008699A61000A033AC0B29A617047C046CC
:102730000008004800040048F7B504000E004D7A78
:10274000C046C046C046C046C046C046C046C04659
:10275000C0460022AA215848FFF79AFF00225521BF
:102760005648FFF795FF2402002220215248FFF728
:102770008FFF23B20193EBB20093337AAB4216D2B0
:102780008020009B0022737290210002FFF780FFDF
:102790000022802011000002FFF77AFF8020002233
:1027A000F0210002FFF774FFC0460020FEBD444B3D
:1027B000444A196808200A43FF211A605A690A40EE
:1027C000A02109020A435A6190220121D205906298
:1027D0009162C046C046C046C046FF2490619161E8
:1027E0001A6839492C400A401A60019B009A1C4320
:1027F0007368A4B2995C20000022FFF749FFC0462D
:10280000C046C046C046C046C046C046C046C04698
:10281000C04600212000FFF76BFF0700C046C046FE
:10282000C046C046C046C046C046C046C0467368A3
:10283000009A9B5C834217D0C046C046C046C04643
:10284000C046C046C046C046C04600212000FFF733
:102850004FFFB8420BD1C046C046C046C046C04636
:10286000C046C046C046C0460135ADB283E7C0464B
:10287000C046C046C046C046C046C046C046C04628
:10288000C046C046C046C046C046C046C046C04618
:10289000C046C046C046C046C046C046C046C04608
:1028A000C046C046C046C046C04600212000FFF7D3
:1028B0001FFF0700C9E7C046AA8A0000558500002F
:1028C0000004004800005555FFFFAAAA70B5040097
:1028D0000D000022AA210F48FFF7DAFE0022552141
:1028E0000D48FFF7D5FE0022A0210A48FFF7D0FED1
:1028F000002229002000FFF7CBFE00212000FFF777
:10290000F7FE0500C04600212000FFF7F1FEA842B7
:10291000F3D170BDAA8A00005585000070B504008F
:102920000D000022AA210F48FFF7B2FE0022552118
:102930000D48FFF7ADFE0022A0210A48FFF7A8FED0
:10294000002229002000FFF7A3FE00212000FFF74E
:10295000CFFE0500C04600212000FFF7C9FEA842B7
:10296000F3D170BD55550000AA2A0000C9015208D4
:102970000A43FF21F0B585B00293234B0500586947
:1029800012B209021140C0B20143902459610121E1
:10299000E405A1620331A162FF213F2658690902C3
:1029A000D2B2084010435861B4460020174F01933B
:1029B0000391C046C046C046C046C046C046C04659
:1029C000C0466346396926698908F6089E4319405E
:1029D000314329543E69411C019BC9B2360A6E54E9
:1029E0005969039B01321940D2B2019B11435961CD
:1029F0000230029BC0B28342DBD20423A361033BBB
:102A0000A36105B0F0BDC0460008004800040048BE
:102A10000F4B30B59022586180230124D205DB0092
:102A200093620C4B94621D680B480902284318609E
:102A30005869C0B201435961C04608219162C0463D
:102A400091611968054801401960946130BDC04624
:102A5000000800480004004800005555FFFFAAAADE
:102A60000B4B10B580215861902301220424DB0513
:102A7000C90099619A629C62C046C046C04605483A
:102A800000699C61000A9962C0B29A6110BDC0469B
:102A900000080048000400480E4B984202D88023EA
:102AA0001B0218430C4B0D4A58610D4B0902186864
:102AB00002431A605A69D2B211435961C04690224A
:102AC0000821D2059162C04691611A6805490A4001
:102AD0001A607047FF1F00000008004800005555AD
:102AE00000040048FFFFAAAA0A4B984202D880239C
:102AF0001B021843084B042258619023DB059A629D
:102B0000C046C046C046C046044908699A61000AEA
:102B1000C0B27047FF1F00000008004800040048D2
:102B200070B504000D000D48AA21FFF7B5FF55212F
:102B30000B48FFF7B1FFA0210848FFF7ADFF2900C0
:102B40002000FFF7A9FF2000FFF7CEFF0500C046D9
:102B50002000FFF7C9FFA842F5D170BD5515000050
:102B6000AA1A000070B504000D000D48AA21FFF755
:102B700093FF55210B48FFF78FFFA0210848FFF76F
:102B80008BFF29002000FFF787FF2000FFF7ACFF35
:102B90000500C0462000FFF7A7FFA842F5D170BD91
:102BA00055150000AA0A00009023DB0530B51C680B
:102BB000134D09022C401C60DA68124C2A40DA607E
:102BC000114A506102229A62104A00B215682C43E1
:102BD00014605469E4B2214351618021C9009961B4
:102BE000002801DA01209862C046C046996201219E
:102BF000996149189961136805490B40136030BD0C
:102C0000FFEFFFFF00005555000800480004004892
:102C1000FFFFAAAAF7B51C4B07001D781B4B0191BB
:102C20001C88202126002036B6B23000FFF7BCFFFA
:102C3000AA211748FFF730FF2000103080B2102182
:102C4000FFF7B2FF2D0155211248FFF725FFEDB226
:102C500020213000FFF7A8FF6419A0210C48FFF7DE
:102C60001BFFA0B22900FFF79FFF01993800FFF773
:102C700013FF3800FFF738FF0400C0463800FFF7A5
:102C800033FFA042F5D1F7BD8C04002036040020AC
:102C900055150000AA0A000070B50400B0200E000F
:102CA00000020A21FFF780FFC0200A210002FFF77F
:102CB0007BFFAA211248FFF7EFFE55211148FFF7CD
:102CC000EBFEA0210E48FFF7E7FEB0200E4B0002FE
:102CD0001D782900FFF768FFC02029000002FFF7D8
:102CE00063FF31002000FFF7D7FE2000FFF7FCFE56
:102CF0000500C0462000FFF7F7FEA842F5D170BDE1
:102D000055150000AA0A00008C040020F8B5050043
:102D10000E00194B02211C88A71CBFB23800FFF718
:102D200043FFAA211548FFF7B7FE601C80B20121BE
:102D3000FFF73AFF55211248FFF7AEFE0221380097
:102D4000FFF732FFA0210D48FFF7A6FE0D4B1978C3
:102D50006418A0B2FFF728FF31002800FFF79CFE9F
:102D60002800FFF7C1FE0400C0462800FFF7BCFEA4
:102D7000A042F5D1F8BDC04636040020551500002C
:102D8000AA0A00008C0400200D4B80225861902379
:102D9000D200DB0500B29A61002801DA01229A62B2
:102DA000C046C046C046C046064B802218699023E4
:102DB000D200DB059A620122000AC0B29A61704714
:102DC000000800480004004870B50400C0200D0051
:102DD00000020121FFF7E8FEAA211548FFF7E4FEF3
:102DE000C02000210002FFF7DFFE55211148FFF748
:102DF000DBFEC02001210002FFF7D6FEA0210C4817
:102E0000FFF7D2FEC0200C4B00021978FFF7CCFE72
:102E100029002000FFF7C8FE2000FFF7B5FF0500DE
:102E2000C0462000FFF7B0FFA842F5D170BDC046F4
:102E300055950000AAAA00008C04002070B504007B
:102E40000D001048AA21FFF7AFFE55210E48FFF7ED
:102E5000ABFEA0210B48FFF7A7FE29002000FFF7DB
:102E6000A3FEA020094B00021978FFF79DFE200069
:102E7000FFF78AFF0500C0462000FFF785FFA84244
:102E8000F5D170BDAAFA000055F500008C040020B1
:102E900070B504000D001048AA21FFF785FE5521EA
:102EA0000E48FFF781FEA0210B48FFF77DFE2900A9
:102EB0002000FFF779FE802000210002FFF774FE5A
:102EC0002000FFF761FF0500C0462000FFF75CFF10
:102ED000A842F5D170BDC04655D50000AAAA000091
:102EE0000D4B0E4A58610E4B0902186802431A60D6
:102EF0005A69D2B21143902259618021D2051068DB
:102F00004901014311604021916291611A680549AC
:102F10000A401A607047C046000800480000555536
:102F200000040048FFFFAAAA104B114A10B55861CF
:102F30001068104B09020343136053690E4CDBB257
:102F40001943902351618021DB051868490108432A
:102F5000186040209862186820401860D8680143C3
:102F6000D960136805490B40136010BD0008004884
:102F70000004004800005555FFEFFFFFFFFFAAAA1D
:102F800070B505000E00134B00211C882000FFF7D0
:102F90000BFEAA211048FFF7C7FF55210F48FFF786
:102FA000C3FFA0210C48FFF7BFFF0D4B1978641831
:102FB000A0B2FFF7F9FD31002800FFF7B5FF2800A8
:102FC000FFF7E2FE0400C0462800FFF7DDFEA04246
:102FD000F5D170BD3604002055550000AA2A000026
:102FE0008C04002070B504000D000D48AA21FFF7E5
:102FF0009BFF55210B48FFF797FFA0210848FFF7DB
:1030000093FF29002000FFF78FFF2000FFF7BCFE91
:103010000500C0462000FFF7B7FEA842F5D170BDFD
:1030200055550000AA2A0000902270B50225D2054D
:103030009561C046C046C046C046C046C046012451
:10304000094B94611E680949314319600849098890
:103050005961C04695625861C04694621A68054934
:103060000A401A6070BDC0460008004855555555C5
:10307000A0040020AAAAAAAAF0B58BB00992012246
:1030800008911100354B02901F78354B1B78049343
:10309000344B1D68344B1B789940344B01911868B0
:1030A000334BA9621B789A40029B102B4FD182624E
:1030B000012421002F4B05941B6806932E4B1B788F
:1030C00099408BB2210007932C4B1B689C462C4BDC
:1030D0001B789940002303911900029C202C05D1F4
:1030E000049E059C1E41264236D08261089C202CFD
:1030F0000FD1002B01D11A4C6354069C2669079C02
:10310000264206D0164C665C059C9C402643144C17
:103110006654099C013FFFB2002C03D0002F01D15F
:10312000019CAC616446039E0133DBB2A661A662DA
:10313000082B05D101310A4BC9B25B5C0493002313
:10314000002FCAD1019B8262AB620BB0F0BD029B23
:10315000112BADD18261ABE78262C7E7E5040020A5
:10316000C50400202C070020300700201C07002089
:103170002007002024070020280700201407002033
:1031800018070020F7B501221A4B1C781A4B196852
:103190001A4B1B789A40102826D18A6201263500E6
:1031A000174B01961B680093164B1B789D4000231C
:1031B000AC461D0020280DD1134E019F765D1E41A7
:1031C0003E4215D08A610133DBB2082B02D10023C5
:1031D0000135EDB26646009F013CE4B2BE61BE62BD
:1031E000002CE7D18A62F7BD1128D7D18A61D5E7D3
:1031F0008A62E8E7E50400202C0700203007002061
:103200001407002018070020C5040020F0B52C4B3F
:1032100085B01B78019301231E00019A1F00964080
:10322000284A1168284A8E62127802921A0002987F
:10323000824094466046254A126890622448057888
:103240002448AF4000689D408762046803941C00D6
:10325000AC402500039C254305604568019CBD43A7
:1032600045609C401D00A54008681C00284308607C
:103270004868B04348601068029999408C4021002A
:1032800001436046116051688143134851600078E2
:10329000124A984083401268116899431160D168BE
:1032A0000B43D36080220E4B1A70002319000D4A85
:1032B00013700D4A99540133202BFBD105B0F0BD9A
:1032C000300700202C070020200700201C070020CA
:1032D00018070020140700202807002024070020DA
:1032E000E6040020E5040020C504002010B52B4BA7
:1032F0001B78082B4ED013D8294C032B39D006D875
:10330000012B28D0022B2AD0254BEE223AE0062BA7
:103310003AD03DD8042BF7D101222021112021E001
:103320000F2B28D008D81E4C0D2B1FD000220E2B9F
:10333000EAD12021102015E0802B06D0184CFF2B5D
:1033400006D0102BE0D100221FE0FFF75FFF10BD79
:10335000F0232370FBE72020FFF714FF04E0012295
:1033600000212020FFF788FE8223F2E700221100CF
:10337000F7E70122DDE7002220211120FFF77CFE84
:103380008222074B1A70E2E7012220210800E9E7B8
:103390001020E1E71120FFF7F5FEF1E7C40400205B
:1033A000E6040020BC224D4BD203996AF0B50A43D3
:1033B0009A629A6A4A490A409A62B022596952034B
:1033C0000A435A6119009023464ADB051278102AF5
:1033D00003D100221A609A60DA601A684248012418
:1033E00002401A608022D868D2010243DA601A686B
:1033F0003E483F4F02401A608022D8685203024381
:103400000420DA601A68A2431A60DA682243DA609C
:103410001A6882431A60DA680243DA6010221D6873
:1034200095431D60DD682A43DA6040221D6895439C
:103430001D60DD682A43DA601A682E4D2A401A6042
:103440008022DD68D2042A43DA601A682A4D2A40B5
:103450001A608022DD68D2052A43DA601A68274D97
:103460002A4080251A60DA68ED022A43DA60244A8D
:103470001668A6431660D6683443D4601E683E4082
:103480001E60DC683C40DC6080234C691B032343E6
:103490004B611C4B1C4C1E681C4F26431E601E6853
:1034A0003E401E60DE683443DC604B691D434D6165
:1034B0001368174D2B401360D468164B1C43D4601F
:1034C000116829401160D1680B43D36013688343AE
:1034D0001360D3681843D060F0BDC04600100240AE
:1034E000FFFFA1FF08070020FFBFFFFFFFFFEFFF67
:1034F000FFEFFFFFFFFFFFFBFFFFFFBFFFFFFBFF34
:10350000000400480008004855555555AAAAAAAA23
:10351000FFFFAAAA000055550D480E4A038810B5B2
:103520000D49934202D10A7801320A709022042494
:10353000D205013394620380084B18699461084CEA
:103540000B7862691B02D2B2134380B2636110BD73
:103550008A040020FFFF00008804002000080048C3
:1035600000040048F7B50D00042701924C7A0002D0
:1035700003B2A6B200932B7AB34202D26C7200203F
:10358000FEBD00986B682043195D80B2019B98478F
:103590006B681A5D094B824205D01A683A431A607B
:1035A00002229A61E7E71A680134BA431A60DA68BE
:1035B00001363A43DA60E4B2B6B2DCE70004004810
:1035C000F7B50D001600FF27000203B24C7A0193F5
:1035D0002A7AE3B2A24202D26B720020FEBD200022
:1035E0006A683840D15C019B0134184380B2B0470F
:1035F000A4B2EDE7022907D10F4B104A984218D028
:10360000904209D1180007E0032906D10A4B0B4963
:103610000B4A98420BD1080070470429FCD1064B95
:10362000064A984205D006499042F4D0054A88429D
:10363000E6D11000F0E7C046380400204C0400201A
:10364000600400207404002070B506000D000524FD
:103650003000013CFFF798FBE4B229003000FFF78F
:10366000A3FA6D08002CF3D170BDFFFF70B5040004
:10367000A0200D0000020221FFF7E6FFAA2110485A
:10368000FFF70AFA55210F48FFF706FAA0210C4868
:10369000FFF702FAA0200C4B00021978FFF7D4FFC5
:1036A00029002000FFF7F8F92000FFF71DFA0500B8
:1036B000C0462000FFF718FAA842F5D170BDC046F9
:1036C00055150000AA0A00008C04002070B5040003
:1036D000C0200D0000020521FFF7B6FFAA210D480A
:1036E000FFF762FA55210C48FFF75EFAA02109485E
:1036F000FFF75AFA29002000FFF756FA2000FFF7DB
:1037000043FB0500C0462000FFF73EFBA842F5D171
:1037100070BDC04655550000AAAA0000F7B50123A8
:103720000225294F01923A780091054393400421E4
:10373000A020264E2D049BB229433268C00100F020
:1037400047FE040001283DD13B7809209C400543F9
:103750007830A3B232682900FF3000F039FE04004F
:1037600001282FD13B7832689C402900A3B2002069
:1037700000F02EFE0400012824D1009B180AFEF759
:1037800055FF3B7832689C402900A3B200F020FE30
:103790000400012816D16B461878FEF747FF220077
:1037A0003B7829009A4093B2326800F011FE0198EC
:1037B000FEF73CFF3B7832689C402900A3B200F042
:1037C00007FE0400E0B2FEBD100700200C07002039
:1037D000F7B501230225274F00903A780191054360
:1037E00093400421C020244E2D049BB2294332680B
:1037F000800100F0EDFD0400012838D109231D43AC
:103800003B78C0209C403268A3B22900400000F001
:10381000DFFD040001282AD13B7832689C40290052
:10382000A3B2002000F0D4FD040001281FD1019BA9
:10383000180AFEF7FBFE3B7832689C402900A3B2D1
:1038400000F0C6FD0400012811D16B461879FEF77F
:10385000EDFE22003B789A4093B2009A144309226D
:10386000E1B209041143326800F0B2FD0400A0B2D5
:10387000FEBDC046100700200C070020C74BC84AF9
:10388000F0B51A60C74A8BB01A6002225A60A022B3
:1038900012019A600493049BDB68002BFBD19022F9
:1038A000049BC14912031960C04B186802431A6097
:1038B00080220991920219681142FCD001225968B4
:1038C0000A435A608022596852020A435A60802291
:1038D000596852030A435A608022196852040A4305
:1038E0001A608022920419681142FCD01121B04A5A
:1038F000B04C11605A680E398A43110002220A4303
:103900005A608022196B0A431A638022D969120413
:103910000A43DA61A84BE381BC231B689847A74B95
:103920006382A74B238262B6FFF73CFDF022A54BD2
:103930001A70049B099AA44E1A6032782023110051
:103940009943D2291BD1A149A148C978C37802243F
:10395000FF2904D1FF3B1C00631E9C41E4B29D4B38
:10396000DB78FF2B00D003249B4BDB78FF2B00D0B0
:1039700004249A4B9A4F1C703860D22A56D0337860
:10398000F22B05D10022023B3370954B1B68DA7095
:103990003578D02D00D0D6E1914E3068C378802B99
:1039A00000D0D0E18D4B1978FFF724FE0023306062
:1039B000C570068804004372C07AF5B2103820281A
:1039C00000D9BEE1FCF7D8FD12014A018D01910139
:1039D000BD01BD01BD01BD01BD01BD01BD01BD01F7
:1039E000BD01BD01BD01BD013500420050005500C3
:1039F000580062006900A600BC00C400BD01BD0102
:103A0000BD01BD01BD01BD01CB002100FFF7F2FDED
:103A100001230135EDB2A542F7D3002B00D0386069
:103A200080223B68DA70D0233370A8E70023012599
:103A3000F1E7E17B0F2900D9A6E109013143237A9F
:103A4000A278C9B26068FEF787FD0BE03C23E17BFA
:103A50000A009A4300D097E1237AA278294360684C
:103A6000FEF7B0FD607262E0237AA278E17B294321
:103A7000E8E7E17B3F23EBE7227AE17BA378009242
:103A8000002229436068FEF729FDEBE7E17B227AFB
:103A9000A378294300920122F4E7524BE17B586955
:103AA00029430E02C0B230436568A278277A586174
:103AB000902004266031C005C9B286621E001F290D
:103AC00001D801218162FF205969000201401143A0
:103AD0005961C046444900238C46C046C046C04692
:103AE000C046C046C046C046614609690132090A5F
:103AF000E9547169D2B2014001331143DBB2716103
:103B00009F42EAD290220421D2059161033991614A
:103B100063720CE00025267A67687608FFF7FCFCE4
:103B20000135EDB238800237AE42F7D265722C4BC8
:103B30001B6819889A7A52181A80D822DA7002E122
:103B4000E17B237AA27829436068FEF70FFF89E7BB
:103B5000E17B237A29430131A278FF31F4E7A07891
:103B60002D0228436668277AFFF75EFA1D4A9020E7
:103B7000002304259446C0058562C046C0466246BF
:103B8000116985618AB2120AF2545A1C0233D2B208
:103B9000DBB2B1549F42EFD2BAE7C04600300040DA
:103BA000CCCC000055550000AAAA0000001002402D
:103BB00000200240006000403CA5FFFF41080008D3
:103BC00085080008E6040020A40400204C0400201E
:103BD000380400206004002074040020A2040020A7
:103BE000900400200008004800040048E37B1E2BDE
:103BF0000BD1C020B6092233F1B200029D43FEF77B
:103C0000D3FF237AA278802131E71C2B0FD1A0208B
:103C10008121C001FEF7C8FF8020F609F1B2000241
:103C2000FEF7C2FFA0200021C001FEF7BDFF8021EA
:103C3000E27B49421F2A05D00D43EDB2237AA278D8
:103C40002900FFE67022A02095430D432188C00182
:103C50000909C9B2EDB2FEF7A7FFEFE7E37BFE2B40
:103C600000D064E77609F1B2DE48FEF715FF1F21A8
:103C7000636829409C46DC4B09025A69A678D2B297
:103C80000A43277A80215A619022C900D2059161A6
:103C90000121FF209162033191625A6900020240C2
:103CA00032435A61C0460022D04D0390C046604660
:103CB00029690136090A815459690398F6B201400D
:103CC00001323143D2B259619742EFD2902304219D
:103CD000DB0599618021C9009962012199616272B5
:103CE00025E7237AA2786021C1E6E37B002B20D16F
:103CF0008033F6091D43F3B20293FF20029BBB49B8
:103D00009B004A690340BA48024013434B61C020FC
:103D10009021029BC905C000DB004A690340B548F9
:103D2000024013434B61227AA378290000920022BB
:103D3000A8E6012BE1D140217604760E31430291B1
:103D4000DBE7C323E370AC4B1D78F02D00D00DE30F
:103D5000AA4E3468E378982B00D007E3A84B2000E4
:103D60001978FFF747FC00233060C370E07AE570F4
:103D700010382678042800D9F6E2FCF7FDFB07008E
:103D8000FB0189029102EA00C423DBE7E37B002BFD
:103D900006D130008038C0B29A4A2100FFF7E2FB1A
:103DA000E37B012B06D130008038C0B2964A210057
:103DB000FFF706FCE37B032B06D130008038C0B24E
:103DC000924A2100FFF7FCFBE37B042B06D1300075
:103DD0008038C0B28E4A2100FFF7C4FBE37B0A2B78
:103DE00006D130008038C0B28A4A2100FFF7E8FBD4
:103DF000E37BFD2B15D13F20238830409B090593A1
:103E00006B4680261B7D06430793677ABBB20393FC
:103E100033021BB20893237A039A934200D39FE0A4
:103E20006772E37B1E2B06D130008038C0B27A4A1D
:103E30002100FFF797FBE37B0C2B17D11F203040AD
:103E400080260643C0202588A5216D09EDB2C0015A
:103E5000FEF7AAFE29007148FEF7A6FE677A350232
:103E60003D43237ABB4200D3EDE06772E37B1C2B1A
:103E70003BD1A02023888121DB09DBB2C00105935F
:103E8000FEF792FE802005990002FEF78DFEA0202D
:103E90005421C001FEF788FE677AAA21BBB26048B0
:103EA0000393FEF781FE55215E48FEF77DFE20213B
:103EB0005B48FEF779FE802333431B021BB2079356
:103EC000237A039A934200D3DAE080209021000203
:103ED0006772FEF769FE802000210002FEF764FE93
:103EE0008020F0210002FEF75FFEE37B1F2B30D124
:103EF000A0202188C0010909C9B2FEF755FEAA21F8
:103F00004748657AFEF750FE55214648FEF74CFEBD
:103F100043482021FEF748FE702380209E43404204
:103F2000304340B20302AFB20593237ABB4200D3C1
:103F3000EEE08020902100026572FEF735FE8020C1
:103F400000210002FEF730FE8020F0210002FEF783
:103F50002BFEF4232288E370A37A9B18238005E2CA
:103F600000213148FEF720FEAA213048FEF7B8FFB5
:103F700055212F48FEF7B4FFA0212C48FEF7B0FFD3
:103F80006B46187D2B4B0799C01880B2FEF70CFECC
:103F9000089D63683D43ADB2D95D2800FEF7A0FFE0
:103FA000C0462800FEF7F0FE06902800FEF7ECFE63
:103FB000069B8342F4D163680699DA5D0B4B8A4213
:103FC0003AD1039A1968013292B2039204229143C2
:103FD0001960D96801370A43DA600222FFB29A6297
:103FE00019E7C046FF3F00000008004800040048F1
:103FF00003FF0000FFF90000A4040020900400204B
:10400000A2040020E52F0008CD360008812F00080B
:10401000912E00083D2E0008C92D0008FFFF00006A
:10402000AA8A00005585000069FD00005555000072
:10403000AA2A000069FDFFFF042219680A431A60DA
:1040400002229A61E7E6AA21CF48FEF7ADFD55218D
:10405000CE48FEF7A9FDA021CB48FEF7A5FD636879
:104060002800D95DFEF7A0FDC0462800FEF78CFEB3
:1040700003902800FEF788FE039B8342F4D1F0E60C
:10408000A0205421C001FEF78FFD079DA0213D43D4
:10409000ADB22800FEF788FD63682800D95DFEF701
:1040A00083FDC0462800FEF76FFE06902800FEF74D
:1040B0006BFE069B8342F4D16368069ADB5DB44DC8
:1040C00093420FD1039B2A6801339BB203930423CD
:1040D0009A432A60EA6801371343EB600223FFB278
:1040E000AB62EDE6A0208121C001FEF75DFD8020DE
:1040F00005990002FEF758FDA0205421C001FEF7EB
:1041000053FD04232A6813432B600223AB61D7E6D7
:10411000059EA0212E43B6B23000FEF745FD636830
:104120003000595DFEF740FDC0463000FEF72CFE22
:1041300003903000FEF728FE039B8342F4D16368AE
:1041400003995A5D924B8A420DD104211A680135B8
:104150008A431A60DA6801370A43DA600222EDB254
:10416000BFB29A62E1E604211A680A431A60022289
:104170009A61DAE6E37B002B04D1864A2100300005
:10418000FFF71EFAE37B012B04D1834A21003000A4
:10419000FFF716FAE37B022B04D1804A210030009E
:1041A000FFF70EFAE37B042B04D17D4A2100300097
:1041B000FFF706FAE37B0A2B04D17A4A210030008C
:1041C000FFF7FEF9E37B0B2B04D1774A2100300087
:1041D000FFF7F6F9E37BFE2B00D0BAE6218873489F
:1041E0004909C9B2FEF758FCAA217148657AFEF761
:1041F0000FFC55216F48FEF70BFC6D482021FEF7A0
:1042000007FC1F2030400302AFB20593237ABB4264
:104210000DD2657290210020FEF7FAFB0021080004
:10422000FEF7F6FBF0210020FEF7F2FB91E6059E7B
:10423000A0212E433000FEF7EBFB63683000595D90
:10424000FEF7E6FBC0463000FEF70AFC03903000A4
:10425000FEF706FC039B8342F4D1636803995A5D21
:104260004B4B8A420DD104211A6801358A431A60EA
:10427000DA6801370A43DA600222EDB2BFB29A620D
:10428000C4E704211A680A431A6002229A61BDE752
:1042900030006030484A2100C0B2FFF791F958E67B
:1042A000E37B042B06D130008038C0B2434A2100A2
:1042B000FFF786F9E37B052B04D1404A210030004B
:1042C000FFF77EF9E37B062B06D130008038C0B2C1
:1042D0003B4A2100FFF774F9E37B072B04D1384AEE
:1042E00021003000FFF76CF9E37B002B1CD1FF228B
:1042F00080331E4323882648DB09DBB29D004169D9
:104300002A40304DDB0029400A4342619022C02000
:10431000D205C000516903402B4801400B43536153
:1043200021003000FEF708FAE37B012B00D010E6F5
:104330002388174A5B04580E40230343FF209B0049
:10434000516903401F4801400B4390215361C90547
:104350004B691D4A30001A4080239B0013434B6178
:104360002100FEF7E9F9F4E5C323E370174B1B784E
:10437000F02B01D1FFF7DDFA832B01D0FFF7D9FA3B
:10438000FEF7B4FFFFF7D5FA55D50000AAAA000042
:1043900000040048652B00086D3600080D2D00084C
:1043A000212B0008992C0008152C0008FF3F000065
:1043B000AA0A000055050000A92B00081D290008C5
:1043C000CD28000803FF0000FFF90000E6040020EC
:1043D000F0B5474680B4061C081C000C102801D517
:1043E000162700E004270007000F8046FF20014049
:1043F0005468251C1D439C43F60313850AD5C0460B
:10440000C046C046C046C046C046C04694801383DE
:10441000958002E0012000F081F801390AD4381CAF
:1044200000F07CF8C046948013839580C046C04657
:104430007600E2E7381C013800F070F894801383AE
:104440009580042000F06AF8108A184001D0FF20FF
:1044500061E0C046C046C046C046C046C0469480E3
:104460009580108A184055D001200226B04552D0C0
:104470000921168A1E40FCD1012000F04FF89480DB
:10448000C0469580C04603E0C046C046C046C04610
:10449000948095807600108A1840EFF300804000E9
:1044A000C00F0643381C023800F038F8948095801D
:1044B000022000F033F80139EAD5138594800120F9
:1044C00000F02CF813839580301C80210223994042
:1044D0000E401BD1002341085E4149085E41490856
:1044E0005E4149085E4149085E4149085E4149080C
:1044F0005E4149085E4149085E41760808D340089C
:10450000FF21084048400002013004E00E2002E094
:10451000092000E0002080BCB846F0BD0138FDD184
:104520007047C04603685A0003D45B005B08C0189C
:104530007047802212061343F9E7C046F0B557468C
:104540004E46DE464546E0B5814683B09246002998
:1045500025D04B1E9B46002701935B46FB18DC0FC2
:10456000E4184B466410E5005E193000FFF7DAFFEF
:10457000019B8046A3420BD0280008304844FFF737
:10458000D1FFD04506D80138504509D2671CE4E771
:10459000504505D9A74202D0631E9B46DDE70026A1
:1045A000300003B03CBC90469946A246AB46F0BDF5
:1045B000012809D0022805D0002801D0002070472A
:1045C0000248FCE70248FAE70248F8E7A54C000871
:1045D000BD4C0008B14C000830B5234B83B005003A
:1045E0008C1E002B26D001A9200000E000BF00286F
:1045F0001CD001992200FFF7A1FF041E16D0FFF77F
:1046000091FF6368A864012B2AD0201D002B23DBB7
:10461000FFF788FF0023E8642B650368002B0FDB9E
:10462000FFF780FF2861002003B030BD0023092080
:104630002B61F9E70D480E49091AC9100191D9E714
:104640001801000FFFF7B4FF2861431E98410823AB
:10465000404298430930E7E70123E8642B65DCE733
:10466000002305202B61DFE700000000A0550008B3
:1046700070560008036810B50400DA0705D4483006
:104680009B070ED500F06CFC23685A070ED51A075D
:1046900013D5DB0604D42000D130FF3000F06CFCD1
:1046A00010BD00F059FC23685A07F0D42000D03028
:1046B00000F05AFC23681A07EBD420005130FF3079
:1046C00000F056FC2368E4E70368002B00D01B18B9
:1046D00018007047092070477047C04670B5040045
:1046E0000D0008E02B6C2A00636121000120236982
:1046F0009847082807D1296C2000FFF76DFF002894
:10470000F0D000F083FE0728FBD10020296CFFF7D2
:10471000E3FF281D00F00AFCF0B5CE46474680B501
:10472000C3682E4C9846A5448369060014000431E2
:10473000402205A8994600F071FE002304AD0493C1
:1047400023E0F0222B6C5200736129007CA800F05A
:1047500065FE7CAA31003369200098478A9B0700D8
:104760006B6403934B4600950193320033002100A4
:104770000120C04700281FD1F0227CA95200280048
:1047800000F04CFE0024082F1FD1296C3000FFF7E9
:1047900023FF611E8C41070009340028D1D0AB6B88
:1047A00010216B644B462143019300953300320086
:1047B0000120C047002800D009273800F5239B00BE
:1047C0009D440CBC90469946F0BD072FF4D12000C3
:1047D000296CFFF781FF05A800F0A8FB2CFCFFFF68
:1047E000406C704770B5CB6BFAB00B6404000E00E0
:1047F0004022043103A800F011FE01235B42029322
:1048000006E002AA210023699847050008280AD17A
:10481000129B200019000193FFF7DEFE0028F0D064
:1048200009207AB070BD02A8FFF724FF062DF7D14A
:1048300031002000FFF752FF10B58261DA6BC160D2
:104840001A6419000022FFF767FF10BD436970B5B5
:104850000B64C36804000D00002B15D10A00236906
:10486000010002209847072807D0082803D1290013
:104870002000FFF733FF00F0C9FD0020296CFFF78F
:104880002BFF281D00F052FB0122FFF745FF00F02F
:10489000BDFDC046C36810B5002B05D0CB6B002210
:1048A0000B64FFF739FF10BDFFF79CFFFBE7C04625
:1048B0007047C046836810B5002B02D0010001206C
:1048C000984710BD012906D0002906D003390220DF
:1048D000012900D970470120FCE7002B08D10F2ADD
:1048E00006D8920082185268009B00201A60F1E7F7
:1048F0000220EFE700B585B003AB0A00009300216A
:104900000023FFF7DFFF039805B000BD012906D0A3
:10491000002906D003390220012900D9704701205F
:10492000FCE7002B08D10F2A06D8009B92001B68D9
:10493000821853600020F1E70220EFE700B585B050
:1049400003AB039200930A0000230021FFF7DEFF70
:1049500005B000BD70B51A4CD36BA54413640600B6
:104960000D0019A8111D402200F058FD01235B42E3
:10497000189314E00C2118A802AAFFF7DFFF290002
:1049800018A8B047002812D1069B18AA02A908301F
:1049900001939847040005280AD0092807D0289BCE
:1049A00002A819000193FFF717FE0028E2D009249E
:1049B00018A8FFF75FFE200090239B009D4470BD68
:1049C000C0FDFFFFF0B5DE4657464E464546E0B512
:1049D000160003220D0011008BB01F000193EB6C39
:1049E00001401C1D009107A91B688B460894002FED
:1049F0006BD01A0C1B045946079302230B72FD332C
:104A000013409B004A72E418009B022B00D1AC6B50
:104A10002B6DDB0747D40023059308330340029333
:104A20002768002F00D112E1019B022B49D0638837
:104A3000278898460434012340469A469843AB6C35
:104A40000F21994681443000FFF754FF0021814532
:104A500006D839005346994349448842894149421E
:104A600043465A0002231340012217403B43012BC7
:104A70003AD0002B30D0022B1BD12368009A5F0064
:104A80007F08002A67D1002906D0029A002A00D1A7
:104A90007CE0002F00D1A9E0002B00DA04340137BC
:104AA000BF00E419BCE75946300000F00BFB0028BA
:104AB00010D009200BB03CBC90469946A246AB46AC
:104AC000F0BD636808349846B5E71B0207935B4660
:104AD0001A8199E70820EDE7009B002B02D00029FE
:104AE00000D08DE004349BE7009B002B1AD10029F5
:104AF00016D02368DF0F63689A1CDAD02A00583278
:104B00000692013300D1BDE0201DFFF7DDFD06ABAD
:104B100001003A00280000E000BF002800D082E039
:104B200008347DE70D2130002F6AFFF7E3FE87424E
:104B3000F6D1AB6A9C42F3D12000FFF7F3FC0F21C2
:104B400002003000FFF7FAFE30002A000021FFF7D4
:104B5000F5FE0720AEE72B6A0D2130009846FFF7DF
:104B6000C9FE804501D0236896E7AB6A9C42FAD122
:104B70000023EB6204332B63231DAF626B63236856
:104B8000002B00DA86E00123059388E7002F2DD063
:104B900058239C46AC4463460393231D9946002347
:104BA000984606AB220004933B004C464746B2466B
:104BB00098462E00914603E004342F00454542D02C
:104BC000039B20000693FFF77FFD049B010000225A
:104BD00030007D1C00E000BF0028EDD04346B84601
:104BE00035004C4656461F009845BCD10D2130007B
:104BF000FFF780FE069B28626B62AC62062059E7D5
:104C00002000FFF78FFC04340700AC63280000E0AD
:104C100000BF002800D14CE730003A000F21FFF719
:104C20008DFE072046E707000D213000FFF762FEEA
:104C30002862022F2BD1069BEB622B002C336B6278
:104C4000AC62062036E735004C465646CEE759465C
:104C5000300000F037FA002800D02AE7059B002B2F
:104C600000D137E70F213000FFF744FE0E2102008C
:104C70003000FFF763FE3000094A0F21FFF75EFEA8
:104C8000072017E70D213000FFF734FE2862069B4E
:104C90006B62D5E738000130800020184DE7C04630
:104CA0000000000010B50023FFF78CFE10BDC046C9
:104CB00010B50123FFF786FE10BDC04610B50223D4
:104CC000FFF780FE10BDC046F0B5CE46474680B522
:104CD0000500C3B014001E00012955D000294BD097
:104CE000032922D0042949D1002B47D1102A45D8C5
:104CF000102203681A4200D0F1E020AF380000F023
:104D00003DF900230120A96B02009A40144203D010
:104D10000E689A00BE5004310133042BF4D13800E0
:104D2000A96300F029F9002029E0032B26D11404FF
:104D3000230C160C9846F318102B1FD80822036872
:104D40001A4200D098E020AF380000F013F9424634
:104D5000AB6BF6001C00002A08D0D400F21A1C1914
:104D6000BA181968D15004339C42FAD1AC633800A8
:104D700000F0FEF8002002E0002B24D0022043B017
:104D80000CBC90469946F0BD130C14049846240CB4
:104D9000012E2ED0052EF1D11B19202BEED8424624
:104DA0000F2A70D9A146002C7ED1AA6B4346AA6374
:104DB0000F2B00D89AE04B46002BDBD0684600F062
:104DC000D3F80020DBE700231004A96B000C0136A8
:104DD00032009A40104204D00F689A00AA18576017
:104DE00004310133102BF3D10020A304C7D4A963ED
:104DF000C5E71B19102BC1D843460F2BBED82B6813
:104E00001E4206D00322280093432B60483000F056
:104E1000A5F820AF380000F0A1F8AA6B002C24D030
:104E20004346DB00FF180023994664000023A400DA
:104E3000D158F95004339C42FAD14B4612196F46AF
:104E4000002B0FD04046102800D210204B46D9002E
:104E500000231038C0003818D458C4500433994285
:104E6000FAD15218012EA1D120AF04323800AA6322
:104E700000F072F8002082E7934303605130FF3066
:104E800000F078F85FE7102B3BD910225242914690
:104E900099442B68194208D0022228008B431343FF
:104EA0002B60483000F05EF82B6804221A4221D1B2
:104EB00043460F2B03D820AF380000F053F86F465D
:104EC000380000F053F810244346AA6BE41A002C73
:104ED000B8DD434620AFDB006400FF18A6E793432C
:104EE0000360D130FF3000F049F806E720A800F059
:104EF00037F860E7280093432B60D03000F036F895
:104F0000D6E72B680B4207D0022228008B431343BD
:104F10002B60483000F026F820AF380000F022F86F
:104F2000A146AA6B002C00D07AE73FE7011C343180
:104F300038C9043B9C461D60A646011C20313CC973
:104F400090469946A246AB46011C0831FCC941680F
:104F50000068E54600BDC0467047C0467047C04681
:104F60007047C0467047C0467047C0467047C0464D
:104F70007047C0467047C0467047C0467047C0463D
:104F800001B401A801B585B0FFB408A841464A465E
:104F900053465C4665463EC001A83EC80F98009047
:104FA00000230CB401A9FFF71DFC109B12B0184799
:104FB00001B401A801B585B0FFB408A841464A462E
:104FC00053465C4665463EC001A83EC80F98009017
:104FD00000230CB401A9FFF739FC109B12B018474D
:104FE00001B401A801B585B0FFB408A841464A46FE
:104FF00053465C4665463EC001A83EC80F980090E7
:1050000000230CB401A9FFF745FC109B12B0184710
:1050100001B401A801B585B0FFB408A841464A46CD
:1050200053465C4665463EC001A83EC80F980090B6
:1050300000230CB401ABFFF7FFFB109B12B0184725
:1050400001B401A801B585B0FFB408A841464A469D
:1050500053465C4665463EC001A83EC80F98009086
:1050600000230CB401AAFFF775FC109B12B018477F
:10507000027A0300002A0BD1427A002A0FD0013AAB
:1050800042724268111D416003211268017202E000
:10509000013A02720268100E12021A607047B020C4
:1050A000FCE7C04600B585B003AB00930C2200239B
:1050B0000021FFF707FC039805B000BD10B5FFF70E
:1050C000F1FF10BDF0B557464E464546DE4600237B
:1050D000E0B587B003930F339846083B9946802389
:1050E0001B0306000F009A463800FFF7C1FF0400BB
:1050F000B02800D1C3E003062AD5030042469343FB
:10510000DBB2802B00D171E0902B3DD0A02B00D1E1
:1051100085E0B02B50D0C02B00D196E003004A466A
:105120009343DBB2D02B0AD15346024001321A43DB
:10513000052301213000FFF7C7FD0028D4D0092442
:10514000200007B03CBC90469946A246AB46F0BD55
:10515000FF23820013401D1D05AB9B4600930D22CB
:10516000002300213000FFF7ADFB630620D4059B30
:105170009C46654405955B460D2200930021002363
:105180003000FFF7C3FBAFE7833B03400D2BD6D0C6
:1051900005AD02400095002300213000FFF792FB8F
:1051A000009500230D2200213000FFF7AFFB9BE7A5
:1051B000059B5D1B0595DEE7B12874D0B22800D1B0
:1051C000CFE0B32800D184E0FC230340B42BB6D059
:1051D0004A465346024001321A430121012330005E
:1051E000FFF772FD002800D17EE7A8E7040238002F
:1051F000FFF73EFF802520432D02A8429FD00401E7
:105200000005020C002300213000FFF75DFD00289F
:1052100095D12C4200D167E70123039364E7FF2374
:105220004A461B011900824311410A001A40030734
:1052300002D58023DB011A43002300213000FFF751
:1052400043FD002800D14FE779E7C6284CD0C72896
:105250005ED003004A469343DBB2C02B6DD0C82812
:1052600072D0C92800D06AE73800FFF701FFF023A9
:1052700002031B03134042460240013257E7039BDF
:105280000024002B00D05BE705AD00950E22002125
:105290003000FFF717FB009500230F22002130009C
:1052A000FFF734FB4CE73800FFF7E2FE002800D19F
:1052B00045E7030042469343DBB2002B00D03EE7B4
:1052C000020000213000FFF7FFFC002800D10BE7AF
:1052D00035E73800FFF7CCFEF02302031B03134031
:1052E00042460240013277E73800FFF7C1FEF02363
:1052F00002031B0313404246024001321A430323B8
:1053000003213000FFF7E0FC002800D1ECE616E7AF
:105310003800FFF7ADFE021E00D110E70300414642
:105320008B43DBB2002B00D009E704213000FFF7EC
:10533000CBFC002800D1D7E601E74346A0221C4061
:10534000013412032243DAE73800FFF791FE4346A7
:1053500002009A43D2B210321840120301300243C5
:10536000E6E605AB00939B460D22002300213000AA
:10537000FFF7A8FA3800FFF77BFE030618D57F2554
:10538000B03C059B2840A0409C46604405903800F6
:105390000734FFF76DFE0306F3D481217F238900D4
:1053A00003408C46A340059A62449B180593E2E6AD
:1053B0000224F2E7030000B5DB6C85B05A680800F0
:1053C000120201921A0001A908324A6003220A72ED
:1053D000DB794B72FFF776FE05B000BD10B5FFF725
:1053E0006DFE806C10BDC04610B5FFF767FEC26C45
:1053F000D3799B000833D01810BDC04610B500F01B
:1054000005F8C04610B5FFF7F9FFC04610B50620F5
:1054100000F076F8012000F0A5F8C046F0B50F2A9C
:1054200037D90D0005430C000300AD0735D1150039
:10543000103D2D092E013618103627681F60676849
:105440005F60A7689F60E7681034DF601033B34285
:10545000F3D10F2401352D01491914404519032CAE
:105460001DD90023CE58EE500433E61A032EF9D886
:105470000323043CA4080134A4001A402D1909197F
:10548000002A05D00023CC5CEC5401339342FAD1BE
:10549000F0BD0500002AF5D1FAE70500F2E7220089
:1054A000F8E7C04670B505000C001F2922D8B723C5
:1054B0009B00C358002B0ED08A009B181A68002A44
:1054C00009D0012A10D0511C10D0002120001960F1
:1054D0009047002070BD280000F030F82200010045
:1054E000280000F017F8F5E70020F3E71623036023
:1054F0000120EFE71623036001204042EAE7C0469F
:1055000010B5034B01001868FFF7CCFF10BDC04673
:1055100000000020002370B5074C050008001100B2
:10552000236000F017F8431C00D070BD2368002BE7
:10553000FBD02B60F9E7C0463407002010B500F01F
:1055400001F810BD58220120014B40421A607047FB
:105550003407002058220120014B40421A60704756
:1055600034070020FEE7C046F8B5C046F8B5C0468F
:1055700074B20181B0AB308000000000800A01816C
:10558000B0B0ABF0000000003F020181B0AB308052
:105590000000000080060181B0B0ABF00000000008
:1055A00030EEFF7FB0B0B0807CEFFF7F01000000E5
:1055B00028F0FF7FB0A90280BCF0FF7FB0B0A880C8
:1055C00008F1FF7F0100000014F1FF7FB0B0AA8056
:1055D00048F1FF7F9CFFFF7F08F2FF7F0100000082
:1055E00004F2FF7FAA3F398050F2FF7FB0B0A8805D
:1055F0005CF2FF7FB0B0AA809CF2FF7FB0B0A880C1
:10560000B0F2FF7F01000000ACF2FF7FB0B0A880D5
:10561000B4F2FF7F010000003CF3FF7FAA0FB280CD
:10562000A4F3FF7F58FFFF7F7CF6FF7FB0B0A88018
:1056300098F6FF7F54FFFF7FF4F8FF7F0100000022
:1056400064FAFF7F0084048074FAFF7FB0B0A88002
:1056500074FAFF7F40FFFF7F5CFDFF7F00840480C2
:105660007CFDFF7FB0B0A88094FDFF7F01000000AB
:10567000080000200000000000000000F4020020EC
:105680005C030020C40300200000000000000000B4
:10569000000000000000000000000000000000000A
:1056A00000000000000000000000000000000000FA
:1056B00000000000000000000000000000000000EA
:1056C00000000000000000000000000000000000DA
:1056D00000000000000000000000000000000000CA
:1056E00000000000000000000000000000000000BA
:1056F00000000000000000000000000000000000AA
:105700000000000000000000000000000000000099
:105710000000000000000000000000000000000089
:1057200001000000000000000E33CDAB34126DE626
:10573000ECDE05000B00000000000000000000008F
:105740000000000000000000000000000000000059
:105750000000000000000000000000000000000049
:105760000000000000000000000000000000000039
:105770000000000000000000000000000000000029
:0400000508000805E2
:00000001FF
